:020000021000EC
:10F800000C9446FC0C9463FC0C9463FC0C9463FC19
:10F810000C9463FC0C9463FC0C9463FC0C9463FCEC
:10F820000C9463FC0C9463FC0C9463FC0C9463FCDC
:10F830000C9463FC0C9463FC0C9463FC0C9463FCCC
:10F840000C9463FC0C9463FC0C9463FC0C9463FCBC
:10F850000C9463FC0C9463FC0C9463FC0C9463FCAC
:10F860000C9463FC0C9463FC0C9463FC0C9463FC9C
:10F870000C9463FC0C9463FC0C9463FC0C9463FC8C
:10F880000C9463FC0C9463FC0C9463FC11241FBE69
:10F89000CFEFD0E1DEBFCDBF11E0A0E0B1E0E2EFFD
:10F8A000FFEF01E00BBF02C007900D92A030B1073F
:10F8B000D9F712E0A0E0B1E001C01D92A434B10775
:10F8C000E1F70C94CFFF0C9400FC0F93EF93FF93A0
:10F8D00040D0FC01062F36D0FF91EF910F91089593
:10F8E0000F930F921F92EF93FF9333D0FC010B0104
:10F8F00001E028D0FF91EF911F900F900F91089594
:10F900000F930F92EF93FF9324D0FC0160FD60935F
:10F910006800D895802DE395D895902DFF91EF91B3
:10F920000F900F9108950F930F9213D0082E09E0B6
:10F9300009D00F900F9108950F930BD001E102D0E1
:10F940000F910895E199FECF00936800E895FFFFBD
:10F9500000000091680000FDFCCF089589E08093CD
:10F96000990080919A00806180939A0080919A001A
:10F97000886080939A00089580919C00992708954B
:10F9800040E050E04817590750F429EC38E00000F7
:10F990002150304037FFFBCF4F5F5F4FF3CF0895CB
:10F9A00080919B00992780789070089580919A00AB
:10F9B0008F7E80939A0080919A00877F80939A002F
:10F9C00008950E94D6FC80E7809300400C940000CC
:10F9D000089580939C0080919B0086FFFCCF8091CE
:10F9E0009B00806480939B0008950E94D0FC882334
:10F9F000E1F30E94BCFC803219F481E090E00895AC
:10FA000085E10E94E9FC80E090E008950895EF927E
:10FA1000FF920F931F93CF93DF937B01C0E0D0E061
:10FA2000C617D70770F48C010E94D0FC8823E1F33D
:10FA30000E94BCFCF80181938F012196CE15DF0551
:10FA400098F381E090E0DF91CF911F910F91FF90AB
:10FA5000EF90089590E0282F33272138310589F061
:10FA60002238310524F42038310549F00DC0223800
:10FA7000310549F02839310539F493E005C092E0A9
:10FA800003C091E001C092E1892F9927089540E0D9
:10FA900050E0609140017091410146175707E8F42A
:10FAA000E2E4F1E0809142028EBB809142029091AB
:10FAB0004302292F33272FBB019690934302809353
:10FAC000420280818DBBE29AE19AE199FECF4F5FBD
:10FAD0005F4F31964617570728F308950F931F93EA
:10FAE000CF93DF93809142029091430297FF03C02E
:10FAF00081E08BBF01C01BBE00E010E0809140019F
:10FB00009091410108171907D8F4C2E4D1E080911F
:10FB1000420290914302880F991F60E0800F911F6D
:10FB20000E9480FC8883892F992789830E5F1F4F4D
:10FB3000229680914001909141010817190738F3EE
:10FB4000DF91CF911F910F91089580914001909185
:10FB500041010097C1F0E2E4F1E0AC018091420282
:10FB60008EBB8091420290914302292F33272FBBF5
:10FB700001969093430280934202E09A8DB3819361
:10FB80004150504059F708950F931F93CF93DF933F
:10FB90008C016115710541F0EB01F80181918F0134
:10FBA0000E94E9FC2197C9F781E090E0DF91CF91B5
:10FBB0001F910F9108950F931F93CF93DF93C0E090
:10FBC000D0E00FEF11E0D0934302C0934202D7FF81
:10FBD00003C081E08BBF01C01BBE809142029091A7
:10FBE000430263E0880F991F0E9465FC015010409A
:10FBF000C058DF4F17FFE7CF0E949CFCDF91CF91E9
:10FC00001F910F910895EF92FF920F931F93CF933F
:10FC1000DF93809142029091430297FF03C081E0FD
:10FC20008BBF01C01BBE00E010E0809140019091AD
:10FC300041010817190708F048C0EE24FF24E80125
:10FC4000CD5BDE4FF801EE5BFE4FEE0DFF1D4081F8
:10FC5000888122969927382F2227240F311D8091E1
:10FC6000420290914302880F991FB9018E0D9F1D8A
:10FC70000E9470FC82E090E0E80EF91E9FEFE9160A
:10FC8000F10401F3F8F28091420290914302880F4F
:10FC9000991F63E0800F911F0E9465FC80914202D2
:10FCA00090914302880F991F65E0800F911F0E9479
:10FCB00065FC0E949CFC00501F4F80914001909178
:10FCC00041010817190708F4B8CFDF91CF911F91B0
:10FCD0000F91FF90EF9008951F93CF9310E0C0E233
:10FCE000C093004069E081E090E00E9480FC84FFC6
:10FCF00003C08F7E0E9493FC0E94D0FC8823E1F316
:10FD00000E94BCFC90E6C927C09300409927823529
:10FD10009105DCF4803591050CF054C081349105D7
:10FD200009F45AC0823491053CF48033910509F4FA
:10FD300049C0C19759F12FC18234910509F45FC0C0
:10FD40008534910509F45EC026C18635910509F414
:10FD5000EDC0873591054CF48235910509F461C0F9
:10FD60008535910509F465C016C18437910509F4FC
:10FD7000A0C0853791052CF48436910509F472C032
:10FD80000AC18537910509F4C1C005C10E94F5FC7F
:10FD9000882309F4B1CF84E10E94E9FC81E40E9448
:10FDA000E9FC86E50E94E9FC82E50E94E9FC80E22C
:10FDB0000E94E9FC83E50E94E9FC84E50E94E9FCDD
:10FDC0008BE406C00E94F5FC882309F495CF84E1FA
:10FDD0000E94E9FC80E1E0C061E070E080E091E039
:10FDE0000E9407FD0E94F5FC882309F485CF84E179
:10FDF0000E94E9FC809100010E942AFDE9CF64E1A4
:10FE000070E00AC061E070E080E091E00E9407FDD0
:10FE1000809100019927BC0180E091E00E9407FDDC
:10FE2000D1CF0E94F5FC882309F466CF0E94DBFD48
:10FE3000CECF62E070E080E091E00E9407FD0E947A
:10FE4000F5FC882309F458CF20910001809101012D
:10FE50009927982F8827820F911D909343028093B2
:10FE60004202B5CF63E070E080E091E00E9407FDC0
:10FE700020910101809100019927982F8827820FF6
:10FE8000911D9093410180934001BC0182E491E077
:10FE90000E9407FD0E94F5FC882309F42DCF809174
:10FEA0000201863419F40E9403FE91CF0E9447FD9F
:10FEB0008ECF63E070E080E091E00E9407FD20912A
:10FEC0000101809100019927982F8827820F911DA9
:10FED00090934101809340010E94F5FC882309F42E
:10FEE0000BCF80910201863419F40E946EFD02C08E
:10FEF0000E94A5FD84E10E94E9FC6091400170919F
:10FF0000410182E491E00E94C4FD64CF0E94F5FCAF
:10FF1000882309F4F1CE84E10E94E9FC8EE10E947D
:10FF2000E9FC87E90E94E9FC82E052CF64E070E0DE
:10FF300080E091E00E9407FD0E94F5FC882309F40F
:10FF4000DBCE84E10E94E9FC80910001803531F430
:10FF500080910101882361F4182F17C0883531F48E
:10FF600080910101883061F413E00FC0803531F4D5
:10FF700080910101883049F412E007C0883529F4E6
:10FF800080910101882309F411E069E0812F99270C
:10FF90000E9480FC1DCF85E10E94E9FCADCECFEF31
:10FFA000D0E1DEBFCDBFCEE1F89485B7806885BFD4
:10FFB00080E6809300408D9A959A0E94AEFC0E9444
:10FFC000BCFCCC2361F084E690E00E94C0FC0E945F
:10FFD000D0FC882311F4C150B1F7CC2319F00E9452
:10FFE0006CFE02C00E94E1FC80E090E00C94F8FFFF
:02FFF000FFCF41
:040000031000F800F1
:00000001FF
